:020000020000FC
:1000000000C001E002BB00E007BB00E001BB0FED58
:100010000DBF03E309B9539A549AE8D3809902C0FB
:100020006BD3A9D3E2D3FFD063ECD3D04CD0FBCFBA
:10003000E395C8953196002009F0089550E0DDC0A1
:10004000F3E0EEE6F6DF091679F4F3DF081669F45B
:10005000F0DF071659F43196C895002D3196C895F2
:10006000F02DE02F09950895319631963396EACF19
:1000700090EF80EF21E0088184D0513011F41AD044
:10008000F7CF702F17D00D3091F0952E088179D0D1
:100090000D3069F0951639F4982F872F702F0AD0FC
:1000A0002395233099F708816CD0951609F00895AF
:1000B00001D0F9CFD81529F4C71519F454E09DC023
:1000C0000895CA950895D0E0CFEB0BEA702E8824EE
:1000D000088157D0523009F446C0A5D0A16001C0B4
:1000E000AE7F3DB73B3C12F458E087C0C1DF7D30A6
:1000F000B9F0092D023031F49F708F707F70F5D008
:1001000020D0EFCF9F758F757F75213029F4092D91
:10011000033011F407D0E5CF93DF7D3009F0089567
:10012000A16008957154743012F055E066C078559E
:10013000A0FF11F406D00895F0E0E72F708101D000
:100140000895F0E0E62F70836A956F3B12F456E055
:1001500054C008956395643C12F057E04EC0F0E03F
:10016000E62F70810895F62DE52DE03641F00881E7
:100170000083EA95CA950D30C1F75E2E089552E0CE
:100180003CC0102F1F7555271D3009F415C01030C5
:1001900009F402C01C3011F451E0089510310AF442
:1001A00008951B350AF00895103412F053E00895B5
:1001B0001A310AF452E0089554E00895CF3B19F43F
:1001C00027E02DD00AC0212F33D0C3951DE018831E
:1001D00004C02EE324D0D0E0CFEB2FD0183071F341
:1001E00018831D3049F0CC3A19F427E018D0F5CF28
:1001F000CA95212F1DD0F1CF0895F3E0EEE521D06F
:10020000352F06D00FED0DBF63ECA0E0B0E00BCFB3
:1002100051D0242F04D0232F02D00895202F5D9B8E
:10022000FECF2CB908952DE0FADF2AE0F8DF08951B
:100230002D3011F4F8DF0895F2CF5F9BFECF1CB193
:100240000895C895002021F0202DE9DF3196F9CFDF
:100250000895F7DFE8DF08957DDF07E007174AF02C
:1002600001E0703019F0000F7A95FBCF702F69DF35
:1002700008955AE0C2DF903039F0905D292FCFDF2A
:10028000803011F420E3CBDF803019F0805D282F1F
:10029000C6DF705D272FC3DF08959927882774561E
:1002A00010F09395FCCF7C597A5010F08395FCCFD9
:1002B000765F0895432F4695469546954695405D51
:1002C0004A3308F0495F3F70305D3A3308F0395FD8
:1002D000089546FD475F4F7036FD375F3F70440F0E
:1002E000440F440F440F342B0895882321F00AE073
:1002F000700F8A95D1F7992309F4089504E688943C
:10030000700F9A95C0F751E078CF8DDF8CDFF3E066
:10031000E6E19FDF08954174746F20426173696361
:100320002056302E322E20436F70797269676874C0
:100330002032303032205269636861726420436138
:100340007070656C732C70726F6A65637473406350
:10035000617070656C732E6F72670A0D00004572D4
:10036000726F723D000020204672656500004C49A6
:100370005320440253495A204E024E455720F5035C
:1003800050500B20B50250500D20BC025052494E27
:100390005702505258205E02505242206602505777
:1003A0004D38E10250574520EB0250574F20F702DD
:1003B000454D49549003501A1D20720250501D2083
:1003C0007B02464F52200E034E4558548C02501C5F
:1003D0001E20950250501E20FA0250501C20DB02B5
:1003E00050494620040350544F201003505004201D
:1003F000140352554E20BB03454E44201203414E78
:100400004420C302504F5220CA02454F5220D1020D
:10041000474F544F4203474F535546035245545597
:1004200049035448454E0A034B455920950341431F
:100430004F20A1025341564567034C4F41447C0372
:100440004F5042204F034F44422053035045454BE9
:10045000A602504F4B45AD024F50442057034F4426
:1004600044205C03494E42206003494E442063030C
:10047000534242209D0343424220A403534244205E
:10048000AC0343424420B303CEDEFF27E7EAE51581
:1004900021F02081CDDEEA95FACFC5DEC4DE752DD0
:1004A0007056FBDEE8DEF3E0E6E6D3DE0895AE7FCD
:1004B00018DE50DEF2DEDFDEB6DE089511DE24E265
:1004C000AEDE48DE372FA4DEAEDE089509DE42DE62
:1004D00008E020E3771F08F421E3A1DE0A95C9F7BD
:1004E000A2DE0895AE7FFDDD35DE072F33DEF0E0BE
:1004F000E72F00830895A2FF3FC0AE7FF2DD2ADE22
:10050000A72E28DE872F26DEB72EF0E0E72F808388
:10051000A062A860AA7F0895FF27EB2D00810A152D
:1005200019F003950083A0610895DBDD13DE072F2A
:1005300011DE701719F0772704DE08957FEF01DED2
:10054000089570E0459B71E0FCDD0895C9DD02DE91
:10055000E72FFF277081F5DD0895C2DDFBDD072F52
:10056000F9DDFF27E02F70830895BADDF3DD072F53
:10057000F1DD700FE6DD0895B3DDECDD072FEADD78
:10058000701BDFDD0895ACDDE5DD072FE3DD7023B3
:10059000D8DD0895A5DDDEDD072FDCDD702BD1DD94
:1005A00008959EDDD7DD072FD5DD7027CADD0895BC
:1005B00071E0C7DD089594DDCDDD072FCBDD701729
:1005C0001EC08EDD01E80FBD0EBDBB9AC3DD00E08D
:1005D0000BBD7ABD089584DD03E80FBD01E00EBDBB
:1005E000BB9AB8DD072FB6DD7BBD0ABD089500E0DC
:1005F0000FBD089575DDAEDD072FACDD071770E088
:10060000BAF6B1F29EDD08956BDDA4DD772309F023
:10061000A26008950DB70E5F0DBF0895A460089500
:100620005FDD0895B2600895488144DD388151DE70
:10063000732F87DD3FDD54DD089552DD8BDD472FBD
:10064000FF27E7EA08C05E16DAF400810D3011F0EA
:10065000EA95F9CFEA957727882799275E1682F4DD
:1006600000818FDD523029F4982F872F702FEA9563
:10067000F5CF9F708F707F7038DE471721F7089590
:1006800059E0BBCDDADFDF2FCE2F0895D6DFA06C87
:100690000895B2FF02C0B1600895B260089520DDF0
:1006A00059DD78BB08951CDD55DD77BB089518DD55
:1006B00051DD7E7F72BB089513DD4CDD71BB089563
:1006C00076B33FDD089570B37C7F3BDD089563EC26
:1006D000752D37DD762D35DDDD27C3ECEFE708819D
:1006E000E199FECFEEBB0DBBE29AE19AC03619F05C
:1006F000EA95CA95F4CF0895DD27C3ECEFE7E199B9
:10070000FECFEEBBE09A0DB30883C03619F0EA9530
:10071000CA95F5CF61EC1EDD672E1CDD572E0895BE
:10072000DFDC18DD272F7BDD08955F9BFECF7CB1DA
:10073000733009F4B26005DD0895D2DC8DDD0ADD89
:1007400008B3072B08BB0895CBDC86DD03DD70956D
:1007500008B3072308BB0895C3DC7EDDFBDC02B3CE
:10076000072B02BB0895BCDC77DDF4DC709502B387
:10077000072302BB0895DD27C7EA63EC5F9B04C033
:100780000CB1033009F4B260A5FF03C0CC2EDD2EFE
:10079000AF7DA4FF03C0DD2DCC2DAF7EA6FF03C02F
:1007A000EC2EFD2EAF7BA7FF04C0DF2FCE2FB46051
:1007B000AF77B0FF03C0DF2DCE2DBA7FB1FF03C0EE
:1007C000D62DC52DBD7F5C167AF40881DADCA1FF39
:1007D00004C0543011F0CA95D0CFAD7F523011F41F
:1007E000CA95CBCF7EDCC9CF08958FDD662407EA9A
:1007F000502EF62DE52D63ECA0E0B0E000E008956A
:00000001FF
